:101800004EC083C068C067C066C065C064C063C0A6
:1018100062C061C060C05FC05EC05DC05CC05BC0D4
:101820005AC059C058C00000EC2DFD2DB7B6B0FC11
:10183000FDCF27BFE895B7B6B0FCFDCF21E1B7B625
:10184000B6FCF4CF0895FFFFFFFFFFFF0403090478
:101850001C037700770077002E0066006900730094
:10186000630068006C002E00640065000E035500E4
:101870005300420061007300700012011001FF006C
:101880000008C016DC050201010200010902120075
:101890000101008032090400000000000000112452
:1018A0001FBECFE5D4E0DEBFCDBF10E0A0E6B0E0C4
:1018B000E8EFFFE103C0C89531960D92A836B10755
:1018C000D1F710E0A8E6B0E001C01D92AE39B10733
:1018D000E1F72FD18FC394CFA82FB92F80E090E0EC
:1018E00041E050EA609530E009C02D91822797953C
:1018F000879510F084279527305EC8F36F5FA8F3B3
:101900000895EADF8D939D930895CF93CFB7CF933A
:10191000DF93C395869BE9F7869B0BC0869B09C026
:10192000869B07C0869B05C0869B03C0869B01C023
:1019300089C06F93C0918100DD27C857DF4F2F9377
:1019400065E5869B03C02F916F91E6CF0F931F93A0
:101950004F9320E040E15F9300B3047406FB27F946
:101960003F9350E03BE039C0147440642F77012F5F
:101970005F5F1EC0406810B314742F7752501FC0B1
:10198000406400B32F770474D1F15F5F00C023C0BF
:10199000406210B32F77147491F15F5F00C025C0CF
:1019A00004741027515012F45D5F00001150279508
:1019B0002C3F10B3C8F614740127015027952C3F13
:1019C000C8F64227499300B3047410274F7311508F
:1019D00027952C3FA8F64695469510B3147479F0D8
:1019E0000127015027952C3F98F66B5A60F3315030
:1019F00000B3B0F600C010E41ABF002717C03B5078
:101A00003195C31BD04010E41ABF0881033CF9F0A4
:101A10000B34E9F020917F001981110F1213EDCFE3
:101A2000093651F10D3211F0013E39F7009386006D
:101A30003F915F914F911F910F912F916F91CAB775
:101A4000C6FD67CFDF91CF91CFBFCF911895209181
:101A50008600222369F310918400112339F5343074
:101A60003AF13093840020938000109181003BE094
:101A7000311B309381001CC0009184000130B4F40C
:101A80000AE53091600034FD14C000936000C4E7A3
:101A9000D0E013C0052710E000C0000002BB1AC050
:101AA000052710E0221F1DC010E021C04AE502C03A
:101AB00032ED432FC4E1D0E032E011B31464969AC2
:101AC00002B311BB54E420E865E320FF052702BB05
:101AD000279517951C3FF0F66695B8F7B1F720FFEC
:101AE000052702BB279517951C3FD0F6279517951C
:101AF00017FF052700001C3F02BBB0F629913A955D
:101B000019F70B7B10918500110FC651D04002BB15
:101B100011F010937F0010E41ABF006411B31B7B17
:101B2000402F4B7B54E05A95F1F702BB11BB42BBEF
:101B30007FCF11BA80E882BB14BE81E08BBF82E008
:101B40008BBF879935C288E10FB6F89481BD11BC6F
:101B50000FBE85B7826085BF8BB780648BBF8E9ABE
:101B600020E004C080EA9FE00197F1F72150D1F70F
:101B70008E98789480918400835087FD74C19091F1
:101B80008100CCE0D0E0C91BD109C857DF4F90914C
:101B900080009D3209F0E2C0883009F062C183EC18
:101BA000809374008AE580936000109268004881F9
:101BB000842F80763981882309F463C08EE690E013
:101BC0009093830080938200333081F59B818C81D8
:101BD0002A81203339F48370E82FF0E0ED59FF4F6C
:101BE000808120C0283529F4992371F4E1E0F0E0E8
:101BF00006C0203571F49923A1F4E0E0F0E089E01B
:101C00008093570084910EC0983059F4E3E0F0E0DF
:101C1000F6CF203A11F4D9D105C0203C11F46D81E2
:101C2000DCD180E08093710024E08EC0353029F152
:101C3000832F84508630A8F48A819B8190936A0018
:101C4000809369003930D9F02E8120936B008D810B
:101C5000827080936C0030936D0047FD71C02FEF50
:101C60006FC0323021F4809161008E7F03C080917B
:101C7000610081608093610002C021E065C020E0C6
:101C800063C08A8110927D00332331F410927E006C
:101C90008DE790E022E04FC0353019F48093850045
:101CA00040C03630A9F59B81913019F48AE798E15C
:101CB00004C0923041F48CE898E1909383008093C3
:101CC000820022E121C09330F1F4882341F48CE4B6
:101CD00098E1909383008093820024E015C08130C6
:101CE00041F480E598E190938300809382002CE199
:101CF0000BC0823041F48CE698E19093830080938E
:101D000082002EE001C020E080E4809368001CC0C7
:101D1000383059F0393019F48093870002C03A30D6
:101D200039F08DE790E020E006C087E890E002C03F
:101D30008DE790E021E0909383008093820004C0BF
:101D400080E88093680007C08F81882321F48E810A
:101D5000821708F4282F2093620083C090916800B6
:101D600097FF7FC090916B00F82E981708F4F92E1A
:101D70009F1990936B00EE24E3949111EE248091CF
:101D80006D00873010F420E065C08E010FC0809197
:101D9000690090916A009C012F5F3F4F30936A0069
:101DA00020936900F80161918F0117D1802F8C1B5E
:101DB0008F1568F352C08091690090916A0038E1F4
:101DC0008030930708F04BC02E5FF894E0916900D3
:101DD000F0916A008991999131E00C01309357009C
:101DE000E895112478948091690090916A00029698
:101DF00090936A00809369008F739070009741F010
:101E0000EE2041F12F1530F180916C00882311F103
:101E1000F894E0916900F0916A00329783E0809332
:101E20005700E895789407B600FCFDCFF894E09150
:101E30006900F0916A00329785E080935700E89539
:101E4000789407B600FCFDCFF89481E180935700A9
:101E5000E89578942F1508F4AECFEE2011F010928B
:101E60006200109284008091600084FF7DC08091A8
:101E700062008F3F09F478C0F82E893010F098E0A6
:101E8000F92E8F19809362008091740098E8892759
:101E900080937400FF2009F455C09091680097FF6B
:101EA0002AC080916B008F1508F4F82E8F1980934B
:101EB0006B000F2D10E00B581F4FC5E7D0E017C087
:101EC00020916D008091690090916A00273010F098
:101ED0007CD002C0FC0184918883219680916900A6
:101EE00090916A00019690936A0080936900C017F0
:101EF000D10731F724C0E0918200F09183008F2D4B
:101F0000815096FF0CC090E08A589F4FA5E7B0E043
:101F100024912D933196A817B907D1F70CC0EF0182
:101F200090E08A589F4FA5E7B0E029912D93FE01DC
:101F3000A817B907D1F7F0938300E0938200FF2D33
:101F4000F93060F485E790E06F2DDBDC8F2D8C5F3E
:101F50008C3041F09FEF9093620004C08FEF80932C
:101F600062008EE18093600084E190B3947431F458
:101F70008150D9F71092850010927F008091610006
:101F8000803130F0879B0FC080916100805109C083
:101F9000879909C080916100823028F080916100AA
:101FA00082508093610080916100882309F0E2CD26
:101FB000F8948E9A12BA1BBE15BE81E08BBF1BBE71
:101FC000E0917200F09173000995E199FECF9FBBFB
:101FD0008EBBE09A99278DB30895262FE199FECF05
:101FE0009FBB8EBB2DBB0FB6F894E29AE19A0FBE51
:081FF00001960895F894FFCF5B
:081FF8005AFEFF1E93070000D2
:0400000300001800E1
:00000001FF
